:10000000882AFF3FFF3FFF3FFF00030E8301BA0036
:100010000408B9000A08BB008A0100308B1A0130BD
:10002000F1007108013A031D1F2800300B1901303F
:10003000F1007108013A031D1F2828200B113B080D
:100040008A00390884003A0E8300FF0E7F0E0900F3
:1000500003138312A4032408003A031D0C2A26303C
:10006000A400A5032508003A031D41282830A50057
:100070003E227008A60070227008A7005722700860
:10008000A8002908003A031DAE280130AA02031C6B
:10009000AB0300302B06031D4F2800302A06031D3A
:1000A000AE280130AA000130AB002C08003A031D35
:1000B0005F282D08013A031D5F280130AE002C088F
:1000C000013A031D69282D08063A031D69280130ED
:1000D000AF002C08013A031D73282D08053A031DB3
:1000E00073280130B0002C08013A031D7D282D082B
:1000F000043A031D7D280130B1002C08013A031D8C
:1001000087282D08033A031D87280130B2002C08E8
:10011000013A031D91282D08023A031D9128013050
:10012000B3002C08013A031D9B282D08013A031D3A
:100130009B280130B4002D08003A031DAD282C087F
:10014000003A031DA9283508033A031DA828B60361
:10015000AC280930AD00AC03AE28AD033708033A34
:10016000031DB5280430B700B7280330B70037089F
:10017000033A031DBF282C08B8008511051637085F
:10018000043A031DC7282D08B80085150512FA2862
:1001900006118611061286122229061586110612EC
:1001A00086122229061186150612861222290615A4
:1001B0008615061286122229061186110616861247
:1001C0002229061586110616861222290611861581
:1001D000061686122229061586150616861222296B
:1001E0000611861106128616222906158611061298
:1001F000861622293808003A0319C8283808013A17
:100200000319CD283808023A0319D2283808033ACE
:100210000319D7283808043A0319DC283808053AA6
:100220000319E1283808063A0319E6283808073A7E
:100230000319EB283808083A0319F0283808093A56
:100240000319F528F02906130130A900AF01B10107
:10025000B301B001B201B401AE010130AA00013016
:10026000AB002630A4000330B600AD010630AC0070
:100270002808013A031D3F29A8010130B5000C2AC6
:100280000613A9012F08013A031D4A29AF010430C2
:10029000B5000C2A3108013A031D5229B10105307D
:1002A000B5000C2A3308013A031D5A29B301063060
:1002B000B5000C2A2E08013A031D6229AE01033055
:1002C000B5000C2A2808013A031D6A29A80102304A
:1002D000B5000C2A2608013A031D7129A601B501B3
:1002E0000C2A0C2A06130130A9002708013A031D25
:1002F0007D29A7010130B5000C2A2608013A031D0B
:100300008429A601B5010C2A0C2A0617A901AE0101
:100310003608003A031D8E29B5010C2A2608013A39
:10032000031D9529A601B5010C2A0C2A0617A9015F
:10033000AF013008013A031DA229B0010130B50018
:1003400006130C2A2808013A031DAB29A801023024
:10035000B50006130C2A2608013A031DB329A6018D
:10036000B50106130C2A0C2A0617A901B10132089F
:10037000013A031DC029B2010130B50006130C2A51
:100380002808013A031DC929A8010230B500061347
:100390000C2A2608013A031DD129A601B50106132E
:1003A0000C2A0C2A0617A901B3013408013A031DCF
:1003B000DE29B4010130B50006130C2A2808013AE1
:1003C000031DE729A8010230B50006130C2A2608F0
:1003D000013A031DEF29A601B50106130C2A0C2AC8
:1003E0003508003A031923293508013A0319402931
:1003F0003508023A031972293508033A0319852989
:100400003508043A031996293508053A0319B42921
:100410003508063A0319D229080001300313831264
:10042000AA000130AB002630A4002830A500063019
:10043000AC000030AD000330B7000030B500003034
:10044000A6000030A7000030A8000130A100013054
:10045000A2000130A3000030AE000030AF00003039
:10046000B0000030B1000030B2000030B300003006
:10047000B4000130A9000330B600080000300313B7
:10048000831286180130F1007108A0007108003A4B
:10049000031D532A2108013A031D532A2008A100F5
:1004A0000130F00008002008A100F0010800003031
:1004B00003138312861B0130F1007108A00071083C
:1004C000003A031D6C2A2308013A031D6C2A2008F8
:1004D000A3000130F00008002008A300F00108008C
:1004E0000130031383120605F1007108A0007108A2
:1004F000003A031D842A2208013A031D842A200899
:10050000A2000130F00008002008A200F00108005D
:100510000D228501860107309F0083168101073077
:10052000850083308600831206138101A0308B0082
:10053000982A992AFF3FFF3FFF3FFF3FFF3FFF3FC2
:02400E00223F4F
:00000001FF
